:100000000C9435010C9452010C9452010C94520141
:100010000C9452010C9452010C9452010C94520114
:100020000C9452010C9452010C9452010C94520104
:100030000C94ED110C9452010C9452010C94520149
:100040000C9452010C9450050C94ED170C94021171
:100050000C948C110C9452010C9452010C9452018A
:100060000C9452010C9452010C9452010C945201C4
:100070004570692D4F53442053657276696365005E
:1000800000416B7475656C6C65732053657474699D
:100090006E67000053657474696E67202000004825
:1000A0006F6568656E73656E736F722000004853EC
:1000B000206D697420536368616C74657220000060
:1000C00048656164696E6720486F6C642000004B6E
:1000D0006F6D706173732000004B6F6D706173738F
:1000E0002066697820000047505320416B74697680
:1000F00020000041636873656E6B6F7070656C758E
:100100006E672000004472656872617465206265E4
:1001100067722E2000004665686C65722046433C7D
:100120002D3E4F5344200000556E7465727370610C
:100130006E6E756E672000004B65696E65205365B5
:100140007474696E672D416E7A6569676500005049
:10015000432F425420616B746976000055656265D7
:10016000726E65686D65204C65747A746573205392
:10017000657474696E6700004B65696E652044653F
:10018000766976652D416E7A656967650000504332
:100190002F425420616B7469760000556562657268
:1001A0006E65686D65204C65747A7465732044656E
:1001B0007669636500004F4E00002D2D2D00004430
:1001C000657669636520756E642056657273696F24
:1001D0006E7361626672616765000044656369768B
:1001E0006520202020203D20000046572D566572B6
:1001F00073696F6E203D200000464300004E4300AF
:100200000046432D6F6C6420465700004550492D31
:100210004D656E750050616C0050432F4254004B89
:10022000656E6E756E670052432D42657472696526
:1002300062004550492D5374726F6D0045786974A2
:10024000004F4E002D2D0076767D76767A76767E7E
:1002500076767776767B76767876767C767679762D
:10026000767D76767A76767E760011241FBECFEF85
:10027000D4E0DEBFCDBF11E0A0E0B1E0E8E9F1E3FA
:1002800002C005900D92AA38B107D9F713E0AAE889
:10029000B1E001C01D92A53BB107E1F70E945F01EB
:1002A0000C94CA180C94000082E981BB8FE084BBD7
:1002B000AC9AAD9A8EE28ABBD99ADD9A08951F93C3
:1002C0001092D2011092CE011092D301E199FECF8B
:1002D00080E090E09FBB8EBBE09A8DB3809391014C
:1002E000E199FECF81E090E09FBB8EBBE09A8DB399
:1002F00080930001E199FECF82E090E09FBB8EBB2E
:10030000E09A8DB380939201E199FECF87E190E06E
:100310009FBB8EBBE09A8DB380939F01E199FECF86
:1003200088E190E09FBB8EBBE09A8DB38093B801CB
:10033000E199FECF8AE190E09FBB8EBBE09A8DB33E
:1003400080930901E199FECF89E190E09FBB8EBBCC
:10035000E09A8DB38093B401E199FECF8BE190E0F8
:100360009FBB8EBBE09A8DB38093930120910001D7
:10037000213079F49EE09093030187E0809304019B
:1003800086E88093050120930601909307018CE095
:100390000EC09CE09093030185E0809304018AE401
:1003A0008093050110920601909307018AE08093E3
:1003B00008010E94FC1582E981BB8FE084BBAC9AE6
:1003C000AD9A8EE28ABBD99ADD9A0E944905809146
:1003D0009101813019F40E94FD0F02C00E94ED0FBF
:1003E0007894A89A0E947F040E94B2050E94A509F1
:1003F00080919301882311F00E94E8098091BD014A
:10040000882311F00E9427130E94E8090E94CE1051
:1004100081E08093F00110927F031092ED018093B0
:10042000700214E036C06091700281E04DEE51E040
:1004300021E00E9472098091ED018F5F8093ED01B0
:100440008091ED018A3029F48091ED018F5F8093D6
:10045000ED011093EC0114C08091EC0160917002E9
:100460002091F0014FE753E00E94720980917F03D1
:100470008F5F80937F038091EC018F5F8093EC010D
:100480008091EC01843140F3809170028F5F809302
:100490007002809170028F3030F28091B001813013
:1004A000E1F71092B0010E949C16F7CF782FD998EF
:1004B00027E030E041E050E0DB9800000000000061
:1004C0000000CA01022E02C0880F991F0A94E2F7A9
:1004D000872311F0DA9A01C0DA98000000000000CA
:1004E0000000DB9A000000000000000021503040B6
:1004F0008FEF2F3F380701F727E030E041E050E071
:10050000DB980000000000000000CA01022E02C0BB
:10051000880F991F0A94E2F7862311F0DA9A01C036
:10052000DA980000000000000000DB9A00000000E4
:1005300000000000215030408FEF2F3F380701F7B7
:10054000DB98DA98D99A089584E064E00E94560214
:1005500080E06CE40E94560210928C0180918C0124
:100560008823E1F38CE66AE00E94560285E060E0B1
:100570000E94560208951F938091B401823051F475
:100580000E940D1010928A0180918A018823E1F364
:1005900010928A0182E661E74FEF0E947C10109270
:1005A0008A0110E00DC080918F01813011F40E940A
:1005B000420E80918A01813019F410928A0111E073
:1005C0008091BA01882311F4112369F38091B40159
:1005D000823011F40E945410112309F0D9C0809187
:1005E000A50380930901809195038093B801209120
:1005F000B801E199FECF88E190E09FBB8EBB2DBB97
:100600000FB6F894E29AE19A0FBE20910901E199A0
:10061000FECF8AE190E09FBB8EBB2DBB0FB6F89456
:10062000E29AE19A0FBE82E061E041E850E00E9468
:100630007D0D82E062E044E950E00E947D0D82E0A1
:1006400064E04FE950E00E947D0D82E065E04EEAF3
:1006500050E00E947D0D82E066E040EC50E00E9498
:100660007D0D82E067E04FEC50E00E947D0D82E05E
:1006700068E049ED50E00E947D0D82E069E047EEC0
:1006800050E00E947D0D82E06AE043EF50E00E945E
:100690007D0D82E06BE048E251E00E947D0D4091CB
:1006A000B6015091B70184E162E00E94520D809141
:1006B000B80180FF05C084E164E046EB51E004C06E
:1006C00084E164E04AEB51E00E947D0D8091B80125
:1006D00081FF05C084E165E046EB51E004C084E1A0
:1006E00065E04AEB51E00E947D0D8091B80182FFE8
:1006F00005C084E166E046EB51E004C084E166E0B9
:100700004AEB51E00E947D0D8091B80183FF05C046
:1007100084E167E046EB51E004C084E167E04AEB26
:1007200051E00E947D0D8091B80184FF05C084E1F5
:1007300068E046EB51E004C084E168E04AEB51E038
:100740000E947D0D8091B80185FF05C084E169E0BC
:1007500046EB51E004C084E169E04AEB51E00E94BD
:100760007D0D8091B80186FF05C084E16AE046EB0B
:1007700051E004C084E16AE04AEB51E00E947D0D43
:100780004091A50384E16BE050E00E94520D20C02F
:1007900082E062E041E850E00E947D0D82E065E089
:1007A00046E151E00E947D0DE199FECF88E190E0A5
:1007B0009FBB8EBBE09A8DB380939503E199FECFEA
:1007C0008AE190E09FBB8EBBE09A8DB380930901D4
:1007D00090919503892F81708093BB01892F887038
:1007E0008093BC01892F80728093BD019470909397
:1007F000BE011F9108951F9380918A018823E1F320
:1008000010928A0183E666E740E00E947C1010E0C7
:100810000DC080918F01813011F40E94250E8091CE
:100820008A01813019F410928A0111E08091B5019A
:10083000882311F4112369F3112309F054C082E0D5
:1008400062E04FEB51E00E947D0D82E064E04BEDF1
:1008500051E00E947D0D82E066E04AEE51E00E9488
:100860007D0D8091B401813031F48EE064E049EF78
:1008700051E00E947D0D8091B401823031F48EE010
:1008800064E04DEF51E00E947D0D8091B401843011
:1008900031F48EE064E041E052E00E947D0D409131
:1008A0004C038EE066E050E00E94520D40914D03F3
:1008B00080E166E050E00E94520D40914E0383E1DA
:1008C00066E050E00E94520D2091B401E199FECF04
:1008D00089E190E09FBB8EBB2DBB0FB6F894E29AE6
:1008E000E19A0FBE0AC0E199FECF89E190E09FBB7B
:1008F0008EBBE09A8DB38093B4011F9108950E943E
:10090000A40283E66FE644E60E947C1010928A01FE
:1009100080918A018823E1F387E062E040E750E0BC
:100920000E947D0D0E94B30510928A0180918A0178
:100930008823E1F310928A0180918A018823E1F3F0
:1009400010928A0180918A018823E1F310928A0132
:1009500084E064E00E94560280E06CE40E9456024B
:1009600080919101882319F40E94FB031CC082E04E
:1009700062E048E751E00E947D0D82E064E04EE8CD
:1009800051E00E947D0D82E066E04BE951E00E945B
:100990007D0DE199FECF89E190E09FBB8EBBE09A8F
:1009A0008DB38093B40180918A018823E1F3109282
:1009B0008A0180918A018823E1F310928A0184E000
:1009C00064E00E94560280E06CE40E94560280912E
:1009D0009101882319F40E94BB0226C082E062E0E4
:1009E00048E351E00E947D0D82E064E04FE451E075
:1009F0000E947D0D82E066E04CE551E00E947D0D95
:100A0000E199FECF88E190E09FBB8EBBE09A8DB369
:100A10008093B801E199FECF8AE190E09FBB8EBB45
:100A2000E09A8DB3809309018091B401823029F45A
:100A300083E66FE64AE00E947C108091B401813029
:100A400029F482E664E64AE00E947C1080918A01E3
:100A50008823E1F310928A0180918A018823E1F3CF
:100A600010928A0180918A018823E1F310928A0111
:100A700080918A018823E1F310928A0180918A0192
:100A80008823E1F310928A0184E064E00E94560218
:100A9000089582E083BF82E48EBD8AE089BF089515
:100AA0001F920F920FB60F9211248F939F938091F4
:100AB0008E018F5F80938E0180918E01883449F57D
:100AC00091E090938D0110928E018091A9038F5F28
:100AD0008093A9038091A903843631F41092A9036D
:100AE00090938A0190938B018091A903823319F42A
:100AF00081E080938B018091A8038F5F8093A8038E
:100B00008091A8038A3029F41092A80381E0809391
:100B10008C019F918F910F900FBE0F901F90189591
:100B2000982F80538A3010F020E005C0903311F4E4
:100B30002AE001C0282F892F81548A3110F4292FEF
:100B40002653892F81568A3110F4292F2C539D3238
:100B500011F429E403C09E3209F421E4822F0895A0
:100B600008950895089585E060E00E94560286E0A9
:100B700063E80E94560287E060E90E94560285E021
:100B800060E00E94560286E064E80E94560287E018
:100B900061E90E94560285E060E00E94560286E00C
:100BA00065E80E94560287E062E90E94560285E0ED
:100BB00060E00E94560286E066E80E94560287E0E6
:100BC00063E90E94560285E060E00E94560286E0DA
:100BD00067E80E94560287E064E90E94560285E0B9
:100BE00060E00E94560286E068E80E94560287E0B4
:100BF00065E90E94560285E060E00E94560286E0A8
:100C000069E80E94560287E066E90E94560285E084
:100C100060E00E94560286E06AE80E94560287E081
:100C200067E90E94560285E060E00E94560286E075
:100C300061EA0E94560287E068E90E94560285E058
:100C400060E00E94560286E062EA0E94560287E057
:100C500069E90E94560285E060E00E94560286E043
:100C600063EA0E94560287E06AE90E94560285E024
:100C700060E00E94560286E064EA0E94560287E025
:100C80006BE90E94560285E060E00E94560286E011
:100C900065EA0E94560287E06CE90E94560285E0F0
:100CA00060E00E94560286E066EA0E94560287E0F3
:100CB0006DE90E94560285E060E00E94560286E0DF
:100CC00067EA0E94560287E06EE90E94560285E0BC
:100CD00060E00E94560286E068EA0E94560287E0C1
:100CE0006FE90E94560285E060E00E94560286E0AD
:100CF0006FEB0E94560287E060EA0E94560285E090
:100D000060E00E94560286E060EC0E94560287E096
:100D100061EA0E94560285E060E00E94560286E089
:100D200061EC0E94560287E062EA0E94560285E06A
:100D300060E00E94560286E062EC0E94560287E064
:100D400063EA0E94560285E060E00E94560286E057
:100D500063EC0E94560287E064EA0E94560285E036
:100D600060E00E94560286E064EC0E94560287E032
:100D700065EA0E94560285E060E00E94560286E025
:100D800065EC0E94560287E066EA0E94560285E002
:100D900060E00E94560286E066EC0E94560287E000
:100DA00067EA0E94560285E060E00E94560286E0F3
:100DB0006DED0E94560287E068EA0E94560285E0C7
:100DC00060E00E94560286E06EED0E94560287E0C7
:100DD00069EA0E94560285E060E00E94560286E0C1
:100DE0006FED0E94560287E06AEA0E94560285E093
:100DF00060E00E94560286E060EE0E94560287E0A4
:100E00006BEA0E94560285E060E00E94560286E08E
:100E100061EE0E94560287E06CEA0E94560285E06D
:100E200060E00E94560286E062EE0E94560287E071
:100E30006DEA0E94560285E060E00E94560286E05C
:100E400063EE0E94560287E06EEA0E94560285E039
:100E500060E00E94560286E064EE0E94560287E03F
:100E60006FEA0E94560285E060E00E94560286E02A
:100E70006BEF0E94560287E060EB0E94560285E00D
:100E800060E00E94560286E06CEF0E94560287E006
:100E900061EB0E94560285E060E00E94560286E007
:100EA0006DEF0E94560287E062EB0E94560285E0D9
:100EB00060E00E94560286E06EEF0E94560287E0D4
:100EC00063EB0E94560285E060E00E94560286E0D5
:100ED0006FEF0E94560287E064EB0E94560285E0A5
:100EE00061E00E94560286E060E00E94560287E0C0
:100EF00065EB0E94560285E061E00E94560286E0A2
:100F000061E00E94560287E066EB0E945602089557
:100F1000BF92CF92DF92EF92FF920F931F93CF93E6
:100F2000DF937C01B62E8C0145E0C42ED12CC80E77
:100F3000D91E862F90E0EC01CC0FDD1FC80FD91F02
:100F4000CA5EDE4F0EC085E0612F0E94560286E029
:100F5000602F0E94560287E068810E9456020F5F50
:100F60001F4F0C151D0578F38701065F1F4F8FE09B
:100F700090E0E80EF91E8B2D90E0EC01CC0FDD1F08
:100F8000C80FD91FCA5EDE4F0EC085E0612F0E94D8
:100F9000560286E0602F0E94560287E068810E9418
:100FA00056020F5F1F4F0E151F0578F3DF91CF918B
:100FB0001F910F91FF90EF90DF90CF90BF90089519
:100FC000EF92FF920F931F93CF93DF938C01EC016D
:100FD00055E0E52EF12CE80EF91E0DC085E06D2FD1
:100FE0000E94560286E06C2F0E94560287E060E065
:100FF0000E9456022196CE15DF0580F3E8012A965D
:10100000015F1F4F0DC085E06D2F0E94560286E0E4
:101010006C2F0E94560287E060E00E9456022196E3
:10102000C017D10780F3DF91CF911F910F91FF90EF
:10103000EF9008951F93CF93DF93C0914902D09111
:101040004A02D7FD12C0CE016AE070E00E94B718D4
:10105000182F16952091040130E0CE016AE070E06F
:101060000E94B718261B310918C0EE27FF27EC1B7A
:10107000FD0BCF016AE070E00E94B718182F16959B
:101080001C5F2091040130E02F5F3F4FCF016AE0E9
:1010900070E00E94B718260F311DE90175E0CC0FF2
:1010A000DD1F7A95E1F7220F331FC21BD30B279662
:1010B0008091120190911301C817D90739F08091DE
:1010C0001201909113010E94E00704C08091C101B8
:1010D000811721F0CE01612F0E9488071093C10172
:1010E000D0931301C0931201DF91CF911F91089506
:1010F000CF92DF92EF92FF920F931F93CF93DF93E4
:101100008C01E62E85E0612F0E94560286E0602F5A
:101110000E945602CE2CDD2484E391E0C80ED91E35
:1011200087E0F60160810E945602EEE1EE2EF12C7E
:10113000E00EF11E85E06F2D0E94560286E06E2DB6
:101140000E94560287E0F60160810E945602E80183
:10115000CC54DF4F025F1E4F85E06D2F0E94560278
:1011600086E06C2F0E94560287E0F60160810E94A3
:1011700056026E96C017D10779F7DF91CF911F9174
:101180000F91FF90EF90DF90CF900895EF92FF9234
:101190000F931F93CF93DF937C0185E06F2D0E9407
:1011A000560286E06E2D0E94560287E060E00E94A3
:1011B00056028701025E1F4F85E0612F0E94560292
:1011C00086E0602F0E94560287E060E00E9456028F
:1011D000E701CC54DF4F8701025F1E4F85E06D2F82
:1011E0000E94560286E06C2F0E94560287E060E063
:1011F0000E9456026E96C017D10781F7DF91CF91FA
:101200001F910F91FF90EF9008951F93CF93DF935D
:10121000E0914702F0914802F7FD14C0CF016AE067
:1012200070E00E94B718182F16951C5F8091050179
:10123000C82FD0E0CF016AE070E00E94B718C61B4B
:10124000D10917C0222733272E1B3F0BC9016AE0A3
:1012500070E00E94B718182F169580910501C82FCD
:10126000D0E02196C9016AE070E00E94B718C60F6D
:10127000D11D8091140190911501C817D90739F03B
:1012800080911401909115010E94C60804C08091BC
:10129000C201811721F0CE01612F0E9478081093BE
:1012A000C201D0931501C0931401DF91CF911F911A
:1012B000089585E060E00E94560286E06FEC0E948F
:1012C000560287E06CE80E94560285E061E00E94C9
:1012D000560286E06BE00E94560287E06DE80E94AD
:1012E00056020895EF92FF920F931F93CF93DF93CF
:1012F0007A019EE1699FB0011124680F711D8B0175
:10130000020F111D1092AA03EB0115C085E06D2F8D
:101310000E94560286E06C2F0E9456028091AA031A
:10132000F701E80FF11D60818F5F8093AA0387E0CA
:101330000E9456022196C017D10740F3DF91CF914A
:101340001F910F91FF90EF9008956091030181E04C
:101350004DE051E025E00E9472090895DF93CF939C
:1013600000D000D0CDB7DEB719821A821C82F89463
:1013700030914F027894832F6AE00E949718282FAB
:101380000E949718482F822F0E949718292F832F89
:101390000E949718992319F48AE08C8301C09C83DA
:1013A000222319F48AE08A8301C02A83498385E4D1
:1013B0008B8383E061E0AE014F5F5F4F24E00E94CA
:1013C00072090F900F900F900F90CF91DF910895B9
:1013D000DF93CF9300D000D0CDB7DEB780E2898312
:1013E0009BE09A8381E38B839C8381E061E0AE0183
:1013F0004F5F5F4F21E00E9472098091930181301D
:1014000079F462E0AE014E5F5F4F21E00E94720905
:1014100081E063E0AE014D5F5F4F22E00E94720900
:101420000F900F900F900F90CF91DF910895DF9361
:10143000CF9300D000D00F92CDB7DEB7DE0111966A
:10144000E1E4F1E085E001900D928150E1F76091D7
:1014500004018CE0AE014F5F5F4F25E00E947209EE
:101460000F900F900F900F900F90CF91DF910895F4
:1014700080E06CE40E9456020895809120039091D0
:101480002103843B910554F08091A50390E02091C5
:101490001E0330911F038217930744F08091C3010C
:1014A000882371F481E08093C30108958091C30182
:1014B000181624F480E06CE40E9456021092C301D6
:1014C000089580E062E40E94560208958F929F92F0
:1014D000AF92BF92CF92DF92EF92FF920F931F9342
:1014E000DF93CF93CDB7DEB72F970FB6F894DEBF5B
:1014F0000FBECDBFFE013B9685E0DF011D928A95B0
:10150000E9F780914B0290914C026EE170E00E94ED
:10151000B718CB01019797FF02C080E090E08E01E1
:101520000F5F1F4FB8014AE050E00E946618F801B3
:1015300001900020E9F73197FE2EF01A80E0CF2CC1
:10154000DD24C7FCD094F6E08F2E912C8C0E9D1ECE
:1015500058010BC0F501E00FF11F80810E9490053A
:10156000080D191DF80180838E2D082F10E0E82E3C
:10157000E3940C151D0574F38093AA0385E169E0DB
:10158000AE01455F5F4F25E00E94720989E18F1926
:1015900069E0A4012F2D0E9472092F960FB6F894CE
:1015A000DEBF0FBECDBFCF91DF911F910F91FF9096
:1015B000EF90DF90CF90BF90AF909F908F90089565
:1015C0008F929F92AF92BF92CF92DF92EF92FF9253
:1015D0000F931F93DF93CF93CDB7DEB72E970FB640
:1015E000F894DEBF0FBECDBF19821A821B821C8207
:1015F0008091A8019091A9018E010B5F1F4FB80146
:101600004AE050E00E946618F80101900020E9F7D6
:101610003197FE2EF01A80E0CF2CDD24C7FCD09449
:10162000AAE08A2E912C8C0E9D1E58010BC0F5014C
:10163000E00FF11F80810E949005080D191DF8012F
:1016400080838E2D082F10E0E82EE3940C151D05E5
:1016500074F38093AA0385E166E0AE014F5F5F4FAC
:1016600024E00E94720989E18F1966E0A4012F2D00
:101670000E9472098091A8019091A901181619067B
:1016800064F485E060E00E94560286E062EC0E940D
:10169000560287E06CE80E9456028091A801909162
:1016A000A90197FF0CC085E060E00E94560286E029
:1016B00062EC0E94560287E06DE80E94560280911B
:1016C000A8019091A901892B61F485E060E00E9456
:1016D000560286E062EC0E94560287E060E00E94BB
:1016E00056022E960FB6F894DEBF0FBECDBFCF9137
:1016F000DF911F910F91FF90EF90DF90CF90BF90FF
:10170000AF909F908F9008958F929F92AF92BF92CB
:10171000CF92DF92EF92FF920F931F93DF93CF93BD
:10172000CDB7DEB72B970FB6F894DEBF0FBECDBF97
:10173000DE011196EEE3F1E083E001900D9281501D
:10174000E1F78E010C5F1F4F80911C0390911D03E8
:10175000B8014AE050E00E946618F80101900020AC
:10176000E9F73197FE2EF01A80E0CF2CDD24C7FC7C
:10177000D094B8E08B2E912C8C0E9D1E58010BC07E
:10178000F501E00FF11F80810E949005080D191DE1
:10179000F80180838E2D082F10E0E82EE3940C15BD
:1017A0001D0574F38093AA038DE06EE0AE014F5FD8
:1017B0005F4F23E00E94720980E18F196EE0A4015F
:1017C0002F2D0E9472092B960FB6F894DEBF0FBE24
:1017D000CDBFCF91DF911F910F91FF90EF90DF90E0
:1017E000CF90BF90AF909F908F9008958F929F92CF
:1017F000AF92BF92DF92EF92FF920F931F93DF930E
:10180000CF93CDB7DEB728970FB6F894DEBF0FBEE3
:10181000CDBF19828AE08A8380919A0190919B01C1
:101820008E010D5F1F4FB8014AE050E00E9466181C
:10183000F80101900020E9F73197E01B80E0EE2EDF
:10184000FF24E7FCF094480106E0A02EB12CAC0E7A
:10185000BD1E0BC0F401E00FF11F80810E949005B6
:101860000A0D1B1DF80180838D2D082F10E0D82E46
:10187000D3940E151F0574F38093AA0380919A01E7
:1018800090919B018E010A5F1F4F0A977CF4609133
:10189000030181E0AE014F5F5F4F21E00E947209BA
:1018A0006091030182E0A80121E005C0609103017D
:1018B00081E0A80122E00E94720980919C01909130
:1018C0009D018E010D5F1F4FB8014AE050E00E945C
:1018D0006618F80101900020E9F73197E01B80E0DD
:1018E000EE2EFF24E7FCF094480116E0A12EB12C67
:1018F000AC0EBD1E0BC0F401E00FF11F80810E94F1
:1019000090050A0D1B1DF80180838D2D082F10E016
:10191000D82ED3940E151F0574F38093AA038091DB
:101920009C0190919D018E010A5F1F4F0A977CF4E4
:101930006091030184E0AE014E5F5F4F21E00E94A1
:1019400072096091030185E0A80121E005C0609162
:10195000030184E0A80122E00E94720928960FB6D4
:10196000F894DEBF0FBECDBFCF91DF911F910F91D5
:10197000FF90EF90DF90BF90AF909F908F90089571
:101980000F931F93DF93CF93CDB7DEB72A970FB690
:10199000F894DEBF0FBECDBF8E010F5F1F4FB801A1
:1019A0004AE050E00E946618F80101900020E9F733
:1019B0003197E01B20E0FF27E7FDF095322F3F5FD6
:1019C000822F90E08E179F0714F4232FF7CF2093D8
:1019D000AA032A960FB6F894DEBF0FBECDBFCF91F3
:1019E000DF911F910F910895AF92BF92CF92DF9236
:1019F000EF92FF920F931F93DF93CF93CDB7DEB794
:101A00006E970FB6F894DEBF0FBECDBFB82EA62ED0
:101A1000D42EA42FB52FFD0101900020E9F73197B6
:101A2000CE2EC41A7E010894E11CF11C242F352F00
:101A3000C9018C0108C0F80181918F010E949005B5
:101A4000F70181937F01802F8D198C15A0F38B2DC9
:101A50006A2DAE014F5F5F4F2C2D0E9472096E966A
:101A60000FB6F894DEBF0FBECDBFCF91DF911F91AF
:101A70000F91FF90EF90DF90CF90BF90AF900895BF
:101A800080919201813069F4609106018091D701C3
:101A900087FD8F5F85958195825F48ED51E00E94BB
:101AA000F40C0895EF92FF920F931F93DF93CF935F
:101AB000CDB7DEB764970FB6F894DEBF0FBECDBFCB
:101AC000F82EE62ECA018E010F5F1F4FB8014AE0C3
:101AD00050E00E9466188F2D6E2DA8010E94F40C14
:101AE00064960FB6F894DEBF0FBECDBFCF91DF91E5
:101AF0001F910F91FF90EF900895BF92CF92DF92C8
:101B0000EF92FF920F931F93DF93CF93CDB7DEB782
:101B100064970FB6F894DEBF0FBECDBFC82EB62EA9
:101B2000FA017E010894E11CF11C04C0AE0DBF1D3A
:101B30009C9331968E2F841B9491A82FB0E099230B
:101B4000A9F7AE0DBF1D1C92F70101900020E9F727
:101B50003197DE2EDE18870107C0F80180810E94D0
:101B60009005F80181938F01802F8E198D15A8F3B0
:101B70008C2D6B2DAE014F5F5F4F2D2D0E94720992
:101B800064960FB6F894DEBF0FBECDBFCF91DF9144
:101B90001F910F91FF90EF90DF90CF90BF9008952D
:101BA0001F93CF93DF93EC01A3E0B0E047C0FD01AA
:101BB000EC58FD4F8081FD01EB58FD4F2081422FF5
:101BC00050E04D535040FD01EA58FD4F7081FD013A
:101BD000E958FD4F10819A01F4E035952795FA9563
:101BE000E1F790E0CD97880F991F880F991F282B58
:101BF000392B2883613029F1E72FF0E0FD9734E09D
:101C0000440F551F3A95E1F75070CF019595879590
:101C100095958795482B592B4983623091F01496FE
:101C2000635086E0EE0FFF1F8A95E1F7F070812F79
:101C300090E0CD97E82BF92BEA832396662309F0F1
:101C4000B6CFDF91CF911F910895809176028635AE
:101C5000B1F48091750281568093B4018091B401F2
:101C6000843018F084E08093B4018CE493E06AE05F
:101C700043E02AE00E94D00D81E08093B5011092EC
:101C80008F0108951F931091B401123009F486C09A
:101C9000143009F4DBC0113009F09BC18091760249
:101CA000813581F48BE893E06BE143E02DE20E9403
:101CB000D00D80918B0390E09093B7018093B60193
:101CC0001093BA0180917602843409F082C18AE0CF
:101CD00093E061E443E021E40E94D00D8091200371
:101CE00090912103843B910554F4809194018130BB
:101CF00031F410929401F8940E94FD0F7894809131
:101D0000200390912103843B91057CF08091940104
:101D1000882359F481E080939401F8948091910193
:101D2000882311F40E94ED0F789480910C03909118
:101D30000D0366E170E00E94B7186E5F7F4F7093ED
:101D40004A026093490280910E0390910F0366E16D
:101D500070E00E94B7186A5F7F4F709348026093EB
:101D60004702809116039091170390934C02809341
:101D70004B0280911E0380934F0280912E0290911E
:101D80002F0290934E0280934D0280911C039091FC
:101D90001D0390935202809351021BC180917602E1
:101DA0008F34A9F0813509F014C18BE893E06BE121
:101DB00043E02DE20E94D00D80918B0390E0909340
:101DC000B7018093B60181E08093BA0102C181EF2F
:101DD00091E060E543E02DE20E94D00D8091390250
:101DE000992787FD9095029690934A028093490225
:101DF00080913A02992787FD909506969093480224
:101E00008093470280912C0290912D0290934C0276
:101E100080934B028091320280934F0280912E0278
:101E200090912F0290934E0280934D028091370241
:101E300090913802909352028093510280912B022C
:101E40008093530281E08093B901C3C080917602F0
:101E5000843409F05AC08AE093E061E443E021E46D
:101E60000E94D00D8091200390912103843B910525
:101E700054F480919401813031F410929401F894DB
:101E80000E94FD0F78948091200390912103843B60
:101E900091057CF080919401882359F481E080932E
:101EA0009401F89480919101882311F40E94ED0F20
:101EB000789480910C0390910D0366E170E00E948C
:101EC000B7186E5F7F4F70934A026093490280910A
:101ED0000E0390910F0366E170E00E94B7186A5FED
:101EE0007F4F709348026093470280911603909150
:101EF000170390934C0280934B0280911C039091A6
:101F00001D039093520280935102809176028C348B
:101F100081F481E090E09093B7018093B60181E075
:101F20008093BA018DE893E069E143E02DE20E94DD
:101F3000D00D809176028D3481F482E090E0909310
:101F4000B7018093B60181E08093BA018DE893E0F8
:101F500069E143E02DE20E94D00D809176028E343B
:101F600081F483E090E09093B7018093B60181E023
:101F70008093BA018DE893E069E143E02DE20E948D
:101F8000D00D809176028F3481F484E090E09093BC
:101F9000B7018093B60181E08093BA018DE893E0A8
:101FA00069E143E02DE20E94D00D809176028035F8
:101FB00081F485E090E09093B7018093B60181E0D1
:101FC0008093BA018DE893E069E143E02DE20E943D
:101FD000D00D10928F011F91089582E289B910BC33
:101FE00080B91CBE909A28E92AB996E890BD82EC87
:101FF0008BB921B99CBF82B9089582E289B910BC1E
:1020000080B91CBE88E98AB926E820BD92EC9BB94C
:1020100080E981B92CBF92B90895DF93CF93CDB7F2
:10202000DEB72C970FB6F894DEBF0FBECDBF83E2AC
:10203000898383E68A8385E78B838DE38C838D8315
:102040008E838F83DE011196FD0120E030E0AE012A
:10205000485F5F4F8191280F311DE417F507D1F7D5
:10206000C9019F7046E0959587954A95E1F7835C95
:1020700088872F733070822F835C89878DE08A87F1
:102080009E01255F3F4F8C91159BFECF83B9119622
:10209000A217B307C1F72C960FB6F894DEBF0FBE98
:1020A000CDBFCF91DF910895DF93CF93CDB7DEB74A
:1020B0002C970FB6F894DEBF0FBECDBF8BE189839E
:1020C0008A8385E58B838AEA8C831D82FE013196A3
:1020D0009E012A5F3F4F8081159BFECF83B93196C9
:1020E000E217F307C1F72C960FB6F894DEBF0FBEC8
:1020F000CDBFCF91DF910895DF93CF93CDB7DEB7FA
:102100002A970FB6F894DEBF0FBECDBF93E2998336
:102110008A836B83842F86958695835C8C8350E0BD
:102120004370507064E0440F551F6A95E1F7435CBB
:102130004D838DE38E838F83DE011196FD0120E0B8
:1021400030E0AE01485F5F4F8191280F311DE417E9
:10215000F507D1F7C9019F7056E0959587955A9577
:10216000E1F7835C88872F733070822F835C8987C7
:102170008DE08A879E01255F3F4F8C91159BFECF96
:1021800083B91196A217B307C1F72A960FB6F89430
:10219000DEBF0FBECDBFCF91DF9108955D9BFECF17
:1021A0008DE68CB95D9BFECF8FE68CB95D9BFECF33
:1021B00089E68CB95D9BFECF8EE68CB95D9BFECF28
:1021C0008DE08CB95D9BFECF8EE38CB90895159B95
:1021D000FECF83B908955D9BFECF8CB90895662329
:1021E00059F020E0FC01E20FF11DE0815D9BFECF84
:1021F000ECB92F5F6217B0F708955D9BFECF8EE3B9
:102200008CB908951F920F920FB60F9211242F933D
:102210003F938F939F93AF93BF93EF93FF932CB113
:102220002093AB0385B398E0892785BB5D9BFECFE8
:102230002CB92D3059F080918A03E82FF0E0EF5946
:10224000FC4F20838F5F80938A0359C0E0918A03FB
:10225000F0E0EF59FC4F20831092B1011092B201CF
:102260001092B30120E030E090E03FC02130B9F09F
:10227000213018F02230C1F524C0A32FB0E0AF59AF
:10228000BC4F8C91803211F421E023C0E92FF0E0A3
:102290008C91EE57FC4F80839093B10124C0A32F03
:1022A000B0E0AF59BC4F8C91803211F422E011C0E4
:1022B000E92FF0E08C91EA59FD4F80839093B201B1
:1022C00012C0A32FB0E0AF59BC4F8C91803219F4EB
:1022D00023E090E009C0E92FF0E08C91E95AFD4F2E
:1022E00080839093B3019F5F3F5F80918A03831740
:1022F00008F0BCCF81E08093B00110928A03FF9177
:10230000EF91BF91AF919F918F913F912F910F903E
:102310000FBE0F901F9018951F920F920FB60F923D
:1023200011248F939F93EF93FF9393B19093AC03FA
:102330009D3081F48091C401813061F4AB9810929A
:10234000C40180938F01E0915703F0E0EC58FD4FFA
:1023500090832DC08091C401882319F0813039F514
:1023600014C0933241F480918F01882321F481E0DD
:102370008093C401AB9A1092570380915703E82FC2
:10238000F0E0EC58FD4F90830CC0E0915703F0E073
:10239000EC58FD4F908380915703853930F480913C
:1023A00057038F5F8093570302C01092C401FF91BF
:1023B000EF919F918F910F900FBE0F901F901895E6
:1023C00085B392E0892785BB08959091970191305C
:1023D00019F485B3892785BB08951F920F920FB614
:1023E0000F9211242F933F935F936F937F938F935B
:1023F0009F93AF93BF938091C6019091C701892BA2
:1024000081F484B595B59093CD018093CC018EB5C0
:102410008F7B8EBD81E090E09093C7018093C601D1
:102420003AC084B595B59093CB018093CA012EB57F
:1024300020642EBD2091CC013091CD011092C701B6
:102440001092C601821B930B865698406CE271E095
:102450000E94A3187093C9016093C8016730710589
:1024600034F086E090E09093C9018093C8012091F8
:10247000C8013091C90180910201992787FD90958B
:102480002817390741F0263031052CF4209302013A
:1024900081E080939E01BF91AF919F918F917F9139
:1024A0006F915F913F912F910F900FBE0F901F90F2
:1024B000189580914B0290914C029093A1018093CA
:1024C000A0018091A0019091A1012091A2013091E1
:1024D000A301821B930B9093A5018093A40180918B
:1024E000A0019091A1019093A3018093A20140913A
:1024F000AC015091AD018091A4019091A501E3E060
:10250000880F991FEA95E1F79A0173E0220F331FB4
:102510007A95E1F7241B350B820F931F68E070E07A
:102520000E94B7187093AD016093AC012091AE0189
:102530003091AF014091AC015091AD01C90163E010
:10254000880F991F6A95E1F7821B930B840F951FE3
:1025500068E070E00E94B7187093AF016093AE011D
:102560008091AE019091AF019093A9018093A80151
:102570000E94E00A089508958F929F92BF92CF9291
:10258000DF92EF92FF920F931F93DF93CF93CDB71C
:10259000DEB72B970FB6F894DEBF0FBECDBFDE01BE
:1025A0001196E0E5F1E083E001900D928150E1F7B2
:1025B000809153028E010C5F1F4F90E0B8014AE0FA
:1025C00050E00E946618F80101900020E9F7319769
:1025D000BE2EB01AEE24FF24CB2CDD24C7FCD094F1
:1025E00088E0882E912C8C0E9D1E0DC0F801EE0DFA
:1025F000FF1D80810E949005F401EE0DFF1D808378
:102600000894E11CF11CEC14FD0484F388E161E002
:10261000AE014F5F5F4F23E00E9472098BE18B197F
:1026200061E0A4012B2D0E9472092B960FB6F8943D
:10263000DEBF0FBECDBFCF91DF911F910F91FF90F5
:10264000EF90DF90CF90BF909F908F9008958AE198
:1026500061E04EE451E022E00E947209089583E6B1
:102660006FE644E60E947C10F89428E088E190E050
:102670000FB6F894A89581BD0FBE21BDFFCF1F9363
:102680009D998AC18091CE018F5F8093CE0111E028
:102690001093D0018091CE01853009F081C18091E5
:1026A000D201882309F08CC01093D2011092D3017B
:1026B00084E064E00E94560283E061E048ED51E06E
:1026C0000E94F40C83E063E04CE052E00E947D0D38
:1026D00084E068E00E94560283E065E045E152E054
:1026E0000E947D0D80910001813029F484E165E034
:1026F00041E452E004C084E165E044E452E00E9419
:102700007D0D84E060E00E94560283E066E049E1CE
:1027100052E00E947D0D80919101813029F484E185
:1027200066E041E452E004C084E166E044E452E043
:102730000E947D0D83E067E04FE152E00E947D0D35
:1027400080919201813029F484E167E041E452E014
:1027500004C084E167E044E452E00E947D0D83E020
:1027600068E047E252E00E947D0D80919F01813038
:1027700029F484E168E041E452E004C084E168E0C7
:1027800044E452E00E947D0D83E069E042E352E0C0
:102790000E947D0D80919301813029F484E169E0EC
:1027A00041E452E004C084E169E044E452E00E9464
:1027B0007D0D83E06BE04CE352E00E947D0DEEC0A6
:1027C0008091D301882349F584E068E00E94560295
:1027D00080910001882339F41093000184E165E0C1
:1027E00041E452E006C01092000184E165E044E457
:1027F00052E00E947D0D20910001E199FECF81E021
:1028000090E09FBB8EBB2DBB0FB6F894E29AE19A85
:102810000FBE84E060E00E9456021091D301113097
:1028200049F584E068E00E94560280919101882376
:1028300039F41093910184E166E041E452E006C06E
:102840001092910184E166E044E452E00E947D0D23
:1028500020919101E199FECF80E090E09FBB8EBB7B
:102860002DBB0FB6F894E29AE19A0FBE84E060E0C7
:102870000E9456028091D301823051F584E068E0D5
:102880000E94560280919201882341F481E0809356
:10289000920184E167E041E452E006C010929201A7
:1028A00084E167E044E452E00E947D0D20919201B2
:1028B000E199FECF82E090E09FBB8EBB2DBB0FB6AF
:1028C000F894E29AE19A0FBE84E060E00E9456021A
:1028D0008091D301833051F584E068E00E94560274
:1028E00080919F01882341F481E080939F0184E1DE
:1028F00068E041E452E006C010929F0184E168E084
:1029000044E452E00E947D0D20919F01E199FECFA9
:1029100087E190E09FBB8EBB2DBB0FB6F894E29A87
:10292000E19A0FBE84E060E00E9456028091D301DC
:10293000843049F568E00E94560280919301882313
:1029400041F481E08093930184E169E041E452E045
:1029500006C01092930184E169E044E452E00E94D1
:102960007D0D20919301E199FECF8BE190E09FBB1B
:102970008EBB2DBB0FB6F894E29AE19A0FBE84E0AD
:1029800060E00E9456028091D301853049F4109294
:10299000D2010E942F1304C01092CE011092D001D8
:1029A0009C9913C19091D201913009F014C1909378
:1029B000D1018091CF018F5F8093CF012091CF0112
:1029C000253009F008C11092CF018091D3018230E7
:1029D00009F469C0833030F4882371F0813009F044
:1029E000FAC035C0843009F4AAC0843008F486C027
:1029F000853009F0F0C0C3C09093D30183E065E057
:102A000045E152E00E947D0D80910001813029F462
:102A100084E165E041E452E004C084E165E044E41F
:102A200052E00E947D0D84E068E00E94560283E03F
:102A300066E049E152E00E947D0D80919101813074
:102A400019F484E166E0B3C084E166E0B5C082E0D9
:102A50008093D30183E066E049E152E00E947D0D5E
:102A600080919101813029F484E166E041E452E0F3
:102A700004C084E166E044E452E00E947D0D84E0FD
:102A800068E00E94560283E067E04FE152E00E9456
:102A90007D0D80919201813019F484E167E087C057
:102AA00084E167E089C083E08093D30167E04FE170
:102AB00052E00E947D0D80919201813029F484E1E1
:102AC00067E041E452E004C084E167E044E452E09E
:102AD0000E947D0D84E068E00E94560283E068E079
:102AE00047E252E00E947D0D80919F01813019F4F0
:102AF00084E168E05CC084E168E05EC084E08093CB
:102B0000D30183E068E047E252E00E947D0D8091AE
:102B10009F01813029F484E168E041E452E004C07F
:102B200084E168E044E452E00E947D0D84E068E0C6
:102B30000E94560283E069E042E352E03FC02093E6
:102B4000D30183E069E042E352E00E947D0D809171
:102B50009301813029F484E169E041E452E004C04A
:102B600084E169E044E452E00E947D0D84E068E085
:102B70000E94560283E06BE04CE352E01FC01092CB
:102B8000D30183E06BE04CE352E00E947D0D84E0D2
:102B900068E00E94560283E065E045E152E00E9451
:102BA0007D0D80910001813029F484E165E041E4EC
:102BB00052E004C084E165E044E452E00E947D0DEF
:102BC00084E060E00E94560206C01092CF0180911E
:102BD000D0018091D1011F910895813061F4E19974
:102BE000FECF80E090E09FBB8EBB6DBB0FB6F8942C
:102BF000E29AE19A0FBE0895DF93CF93CDB7DEB787
:102C000064970FB6F894DEBF0FBECDBF20E0BE01C3
:102C10006F5F7F4F422F50E0E199FECF822F90E00F
:102C20008D5F9F4F9FBB8EBBE09A8DB3FB01E40F7E
:102C3000F51F80838823A9F08F3F11F4108211C003
:102C40002F5FE8CFFD01E852FE4FA40FB51F8C9116
:102C5000808311829F5FA92FB0E0A217B30794F37E
:102C600012C0DE011196FD0101900020E9F73197B5
:102C7000EA1BFB0BE093D70190E02E2F332727FDB3
:102C80003095AD01E8CF64960FB6F894DEBF0FBE65
:102C9000CDBFCF91DF910895DF93CF93CDB7DEB74E
:102CA00060970FB6F894DEBF0FBECDBF8091510282
:102CB00090915202909373028093720280917202FB
:102CC000909173026FE070E00E94A318DE011596E8
:102CD000AD016A1B9E01205F3F4FE62FEA0FF0E037
:102CE000E95BFD4FE491ED93A217B307B1F7609153
:102CF000070119821A821B821C8289E02BE00E9444
:102D00007209609108018EE0AE014F5F5F4F24E0D1
:102D10000E94720960910801409172025091730201
:102D20008FE00E94520D60960FB6F894DEBF0FBE82
:102D3000CDBFCF91DF910895DF93CF93CDB7DEB7AD
:102D4000E4970FB6F894DEBF0FBECDBFDE01179635
:102D5000E3E5F1E087E001900D928150E1F7DE01BB
:102D60001E96EAE5F1E089E001900D928150E1F7CD
:102D7000DE015796E3E6F1E08EE001900D9281507E
:102D8000E1F7DE011196E1E7F1E086E001900D92B6
:102D90008150E1F7DE019596E7E7F1E080E10190EF
:102DA0000D928150E1F7509182036091830340912D
:102DB00084038091850320E030E0803711F421E026
:102DC00030E080E090E04C3611F481E090E0282380
:102DD000392380E0583609F481E090E0653609F443
:102DE00091E0892390E028233923232B79F0CE0129
:102DF000079666E00E94EF10CE010E9668E00E94F2
:102E0000EF10CE0147966DE00E94EF1050918203C3
:102E100060918303409184038091850320E030E03A
:102E2000873711F421E030E080E090E04F3611F474
:102E300081E090E02823392380E0533709F481E0D2
:102E400090E0683609F491E0892390E02823392343
:102E5000232B19F18091660290916702893481F4E5
:102E6000943471F4CE01019665E00E94EF1088ED74
:102E700091E06091D7010E94EF108DE00E94EB106D
:102E80008091660290916702863739F4953629F46D
:102E9000CE01859668E00E94EF1080918203209118
:102EA00083034091840390E0833709F491E080E04C
:102EB000253609F481E09823892F90E020E030E066
:102EC000443711F421E030E082239323892B09F465
:102ED00040C08091660290916702893409F039C040
:102EE000943409F036C020E01CC0A22FB0E0FD01F0
:102EF000E95AFD4FE081E199FECF822F90E08D5F8E
:102F00009F4F9FBB8EBBEDBB0FB6F894E29AE19A40
:102F10000FBEFD01E95AFD4F8081A852BE4F8C9330
:102F20002F5F8091B301281700F3E199FECFE22FC4
:102F3000F0E0CF018D5F9F4F9FBB8EBB1DBA0FB6D8
:102F4000F894E29AE19A0FBEE852FE4F1082209365
:102F5000D701509182036091830340918403809153
:102F6000850320E030E0853611F421E030E080E098
:102F700090E0433711F481E090E02823392380E08A
:102F8000523709F481E090E0653609F491E0892335
:102F900090E028233923232B11F00E942F130E9445
:102FA000FD10E4960FB6F894DEBF0FBECDBFCF91F3
:102FB000DF91089583ED8DB90895813031F461304A
:102FC00011F492980895929A0895823029F461300C
:102FD00011F494980895949A08951F920F920FB641
:102FE0000F9211242F933F934F935F936F937F938F
:102FF0008F939F93AF93BF93EF93FF938091D501EE
:10300000882369F08091D50190E00197E0918801D3
:10301000F0918901E80FF91F8FB1808303C08FB150
:103020008093B4032091D5018091870130E09927E6
:1030300087FD90958217930754F087E08093B30340
:103040001092B1038091D5018093B20309C081E051
:1030500060E00E94DD171092D40181E08093D601D8
:103060008091D5018F5F8093D501FF91EF91BF9142
:10307000AF919F918F917F916F915F914F913F9110
:103080002F910F900FBE0F901F9018951F93182F20
:103090008091D401882311F081E016C0812F61E076
:1030A0000E94DD171093D401113069F486E08093FB
:1030B00087011092D50183E08093B3031092B1038E
:1030C0008AEA8093B20380E01F910895FB019F017B
:1030D000E8944230C4F04532B4F44A3029F497FB06
:1030E0001EF4909581959F4F642F77270E94A31817
:1030F000805D8A330CF0895D8193CB010097A1F745
:1031000016F45DE251931082C9010C948718DC011A
:10311000FC01672F71917723E1F7329704C07C910E
:103120006D9370836291AE17BF07C8F30895991B22
:1031300079E004C0991F961708F0961B881F7A95AE
:10314000C9F780950895AA1BBB1B51E107C0AA1FB0
:10315000BB1FA617B70710F0A61BB70B881F991F38
:103160005A95A9F780959095BC01CD01089597FBDC
:10317000092E07260AD077FD04D0E5DF06D000200F
:103180001AF4709561957F4F0895F6F790958195A3
:083190009F4F0895F894FFCF52
:103198000101030E0786010E0C5C00000A000044C2
:1031A8000000230023005464665363655262005193
:1031B800610050600050600051610052620053632A
:1031C800655464666768696A6B6B6A69686700005A
:1031D8000053536353530A03F1018B030D0A0A1D6D
:1031E80000000068656C70200D0073686F772049D7
:1031F800440D0073686F772076657273696F6E0D82
:10320800004944203D2000302E392E312E302E61C9
:0A3218002E626574610D00085A0370
:00000001FF
